:0400000057EF00F0C6
:10000800D706D706D706D706D706D706D706FE05DA
:10001800D505D706D706D706D706D706D706D706F3
:10002800D706D706D706D706D706D706D706D706E0
:10003800D706D706D706D706D706D706D706A20605
:10004800D706D7063C05D7062B00D706D706D7060E
:10005800D706D706D706D706D706D706D706D706B0
:10006800D706D706D706D706D706D706D706D706A0
:10007800D706D7062B00D706D706D7062B002B00A6
:100088002B002B002B002B002B002B00D706D706AC
:10009800D706D706D706D7062B002B002B002B0038
:0A00A800D706D706FF0016EF0DF093
:1008000000000001E56BE16BE26BE36BE46B20EE53
:1008100069F03B0EDE6AE806FDE220EE78F110EEAC
:10082000A5F03B0E6F006FFFE3FFE806FBE23A0125
:10083000406BC268506BC10EC36EC00E516F606BCF
:10084000C46AD28ED28CD28A39018181D2909181B0
:10085000809F908F3A01568D568FB9501F0B4009DB
:10086000B96EB9980F0EB912FA0EB76EB66AB88E95
:10087000B8983901A39F839F8495060EAE6EAD6A2A
:10088000AF6ACB0EAB6EAA6AA4959485100EAC6EBF
:10089000AC8E4BEC0CF00001E751D8B452EF04F0F1
:1008A00054EF04F083EF05F039019191938FB88EE6
:1008B000000E0001646F010E6AEC09F00001E66BA6
:1008C000E651010FD96EDA6ADF6AE62B3B0EE66568
:1008D0006CEF04F06EEF04F060EF04F0EEEC05F066
:1008E000010E0001EB6FEBC03FF03FC0EDF0EC6B91
:1008F000EE6B4F6A0A0E4E6E6BEC0DF00001E86B6A
:10090000E96BEA6BE951D8B488EF04F08AEF04F0A0
:10091000D7EF04F03C0EEE19D8A491EF04F093EF5A
:1009200004F0AAEF04F0EEC067F0FF0E67276751EE
:10093000A50FD96EDA6ADF50686F6851010FD96E62
:10094000DA6ADF6AEE6BEEC064F0010E6AEC09F061
:10095000D0EF04F0EEC067F0FF0E67276751A50FD8
:10096000D96EDA6ADF50686F6851010FD96EDA6AA2
:10097000DF6AEE2BEEC064F0010E6AEC09F0EEC007
:1009800067F0FF0E000167276751A50FD96EDA6A7D
:10099000DF50686F6851010FD96EDA6A010EDF6EA1
:1009A0004F6A050E4E6E6BEC0DF00001E96BEA51DB
:1009B000D8B4DDEF04F0DFEF04F047EF05F0320EBE
:1009C000EE65E5EF04F0E7EF04F019EF05F0EEC097
:1009D00067F0FF0E67276751A50FD96EDA6ADF50FF
:1009E000686F6851010FD96EDA6ADF6AEEC04EF0A7
:1009F0004F6A516A0A0E506E52EC0BF04E500001D5
:100A0000EE6FEEC064F0010E6AEC09F0EEC067F024
:100A1000FF0E000167276751A50FD96EDA6ADF5014
:100A2000686F6851010FD96EDA6A010EDF6E40EF10
:100A300005F0EEC067F0FF0E67276751A50FD96E6E
:100A4000DA6ADF50686F6851010FD96EDA6ADF6ABF
:100A50000A0EEE27EEC064F0010E6AEC09F0EEC05B
:100A600067F0FF0E000167276751A50FD96EDA6A9C
:100A7000DF50686F6851010FD96EDA6A010EDF6EC0
:100A80004F6A050E4E6E6BEC0DF00001EA6B130E13
:100A9000E8654DEF05F04FEF05F082EF04F0390106
:100AA000939F0001E66BE651690FD96EDA6ADF6A3F
:100AB000E651010FE16EE26A6F007FFFE7FFE62B70
:100AC0003B0EE66566EF05F068EF05F053EF05F0C5
:100AD000000E646F000E6AEC09F0010E0001EC6F6D
:100AE000ECC03FF03FC0EDF0EB6BEEEC05F03901F0
:100AF00091814F6A050E4E6E6BEC0DF00001EA6BB2
:100B0000E76B4BEF04F0E66BE651690FD96EDA6ADA
:100B1000E651010FE16EE26ADE50E618D8B493EFB9
:100B200005F095EF05F0A2EF05F0010EE56FE65137
:100B3000010FD96EDA6AE651690FE16EE26A6F0061
:100B40007FFFE7FFE62B3B0EE665A9EF05F0ABEF75
:100B500005F084EF05F0ED51E119D8B4B2EF05F0DE
:100B6000B4EF05F0B8EF05F0010EE56FEDC0E1F070
:100B7000EC51E219D8B4BFEF05F0C1EF05F0C5EFB5
:100B800005F0010EE56FECC0E2F03F50E319D8B478
:100B9000CCEF05F0CEEF05F0D2EF05F0010EE56FDA
:100BA0003FC0E3F0EB51E419D8B4D9EF05F0DBEF27
:100BB00005F0DFEF05F0010EE56FEBC0E4F0E55165
:100BC000D8B4E5EF05F0E7EF05F04BEF04F0E56B87
:100BD000EEEC05F04BEF04F057EF00F008B002D058
:100BE000BB9A01D0BB8A0CB002D0BB9801D0BB88A5
:100BF0000BB002D0BB9601D0BB860AB002D0BB942A
:100C000001D0BB8409B002D0BB9201D0BB8204B03A
:100C100002D0BC9E01D0BC8E02B002D0BC9C01D0E0
:100C2000BC8C01B002D0BC9A01D0BC8A350EE82E33
:100C3000FED700006F0030FF4EF04E904E924E9463
:100C400060003BF1BCFF350EE82EFED7000003B07C
:100C500002D0BB9A01D0BB8A07B002D0BB9801D0AA
:100C6000BB8806B002D0BB9601D0BB8605B002D0CF
:100C7000BB9401D0BB8426B002D0BB9201D0BB8212
:100C80001BB002D0BC9E01D0BC8E19B002D0BC9C5F
:100C900001D0BC8C15B002D0BC9A01D0BC8A350EF4
:100CA000E82EFED700006F0030FF4EF04E8060004F
:100CB0003BF1BCFF350EE82EFED7000011B002D08C
:100CC000BB9A01D0BB8A12B002D0BB9801D0BB88BE
:100CD00016B002D0BB9601D0BB8617B002D0BB9431
:100CE00001D0BB8418B002D0BB9201D0BB821AB035
:100CF00002D0BC9E01D0BC8E13B002D0BC9C01D0EF
:100D0000BC8C14B002D0BC9A01D0BC8A350EE82E3F
:100D1000FED700006F0030FF4EF04E904E82600014
:100D20003BF1BCFF350EE82EFED7000010B002D01C
:100D3000BB9A01D0BB8A25B002D0BB9801D0BB883A
:100D40001FB002D0BB9601D0BB8620B002D0BB94AE
:100D500001D0BB842AB002D0BB9201D0BB8224B0A8
:100D600002D0BC9E01D0BC8E29B002D0BC9C01D068
:100D7000BC8C27B002D0BC9A01D0BC8A350EE82EBC
:100D8000FED700006F0030FF4EF04E8060003BF158
:100D9000BCFF350EE82EFED7000028B002D0BB9A6B
:100DA00001D0BB8A21B002D0BB9801D0BB8837B03C
:100DB00002D0BB9601D0BB8622B002D0BB9401D03A
:100DC000BB8423B002D0BB9201D0BB8230B002D032
:100DD000BC9E01D0BC8E39B002D0BC9C01D0BC8C72
:100DE00038B002D0BC9A01D0BC8A350EE82EFED7AE
:100DF00000006F0030FF4EF04E904E924E84600027
:100E00003BF1BCFF350EE82EFED700002FB002D01C
:100E1000BB9A01D0BB8A31B002D0BB9801D0BB884D
:100E200036B002D0BB9601D0BB8632B002D0BB94A4
:100E300001D0BB8434B002D0BB9201D0BB8233B0AE
:100E400002D0BC9E01D0BC8E35B002D0BC9C01D07B
:100E5000BC8C2EB002D0BC9A01D0BC8A350EE82ED4
:100E6000FED700006F0030FF4EF04E8060003BF177
:100E7000BCFF350EE82EFED700003AB002D0BB9A78
:100E800001D0BB8A2BB002D0BB9801D0BB880FB079
:100E900002D0BB9601D0BB861EB002D0BB9401D05D
:100EA000BB840EB002D0BB9201D0BB821DB002D079
:100EB000BC9E01D0BC8E0DB002D0BC9C01D0BC8CBD
:100EC0001CB002D0BC9A01D0BC8A350EE82EFED7E9
:100ED00000006F0030FF4EF04E904E8260003BF1FC
:100EE000BCFF350EE82EFED700003CB002D0BB9A06
:100EF00001D0BB8A2DB002D0BB9801D0BB882CB0EA
:100F000002D0BB9601D0BB863BB002D0BB9401D0CF
:100F1000BB840001EDB102D0BB9201D0BB820001C5
:100F2000ECB102D0BC9E01D0BC8E3FB002D0BC9CC4
:100F300001D0BC8C0001EBB102D0BC9A01D0BC8ABC
:100F4000350EE82EFED700006F0030FF4EF04E80C9
:100F500060003BF1BCFF120008B002D0BB9A01D088
:100F6000BB8A0CB002D0BB9801D0BB880BB002D0BA
:100F7000BB9601D0BB860AB002D0BB9401D0BB8423
:100F800009B002D0BB9201D0BB8204B002D0BC9E9B
:100F900001D0BC8E02B002D0BC9C01D0BC8C01B090
:100FA00002D0BC9A01D0BC8A350EE82EFED70000D4
:100FB0006F0030FF45F0459045924594600017F171
:100FC000BCFF350EE82EFED7000003B002D0BB9A5E
:100FD00001D0BB8A07B002D0BB9801D0BB8806B055
:100FE00002D0BB9601D0BB8605B002D0BB9401D025
:100FF000BB8426B002D0BB9201D0BB821BB002D012
:10100000BC9E01D0BC8E19B002D0BC9C01D0BC8C5F
:1010100015B002D0BC9A01D0BC8A350EE82EFED79E
:1010200000006F0030FF45F04580600017F1BCFF05
:10103000350EE82EFED7000011B002D0BB9A01D0C9
:10104000BB8A12B002D0BB9801D0BB8816B002D0C8
:10105000BB9601D0BB8617B002D0BB9401D0BB8435
:1010600018B002D0BB9201D0BB821AB002D0BC9E95
:1010700001D0BC8E13B002D0BC9C01D0BC8C14B08B
:1010800002D0BC9A01D0BC8A350EE82EFED70000F3
:101090006F0030FF45F045904582600017F1BCFFBE
:1010A000350EE82EFED7000010B002D0BB9A01D05A
:1010B000BB8A25B002D0BB9801D0BB881FB002D03C
:1010C000BB9601D0BB8620B002D0BB9401D0BB84BC
:1010D0002AB002D0BB9201D0BB8224B002D0BC9E09
:1010E00001D0BC8E29B002D0BC9C01D0BC8C27B0F2
:1010F00002D0BC9A01D0BC8A350EE82EFED7000083
:101100006F0030FF45F04580600017F1BCFF350EE1
:10111000E82EFED7000028B002D0BB9A01D0BB8ACF
:1011200021B002D0BB9801D0BB8837B002D0BB96AB
:1011300001D0BB8622B002D0BB9401D0BB8423B0C7
:1011400002D0BB9201D0BB8230B002D0BC9E01D095
:10115000BC8E39B002D0BC9C01D0BC8C38B002D05F
:10116000BC9A01D0BC8A350EE82EFED700006F0075
:1011700030FF45F0459045924584600017F1BCFF73
:10118000350EE82EFED700002FB002D0BB9A01D05A
:10119000BB8A31B002D0BB9801D0BB8836B002D038
:1011A000BB9601D0BB8632B002D0BB9401D0BB84C9
:1011B00034B002D0BB9201D0BB8233B002D0BC9E0F
:1011C00001D0BC8E35B002D0BC9C01D0BC8C2EB0FE
:1011D00002D0BC9A01D0BC8A350EE82EFED70000A2
:1011E0006F0030FF45F04580600017F1BCFF350E01
:1011F000E82EFED700003AB002D0BB9A01D0BB8ADD
:101200002BB002D0BB9801D0BB880FB002D0BB96E8
:1012100001D0BB861EB002D0BB9401D0BB840EB0FF
:1012200002D0BB9201D0BB821DB002D0BC9E01D0C7
:10123000BC8E0DB002D0BC9C01D0BC8C1CB002D0C6
:10124000BC9A01D0BC8A350EE82EFED700006F0094
:1012500030FF45F045904582600017F1BCFF350E28
:10126000E82EFED700003CB002D0BB9A01D0BB8A6A
:101270002DB002D0BB9801D0BB882CB002D0BB9659
:1012800001D0BB863BB002D0BB9401D0BB8400012F
:10129000EDB102D0BB9201D0BB820001ECB102D013
:1012A000BC9E01D0BC8E3FB002D0BC9C01D0BC8C97
:1012B0000001EBB102D0BC9A01D0BC8A350EE82EF9
:1012C000FED700006F0030FF45F04580600017F149
:1012D000BCFF12000001656FBC96350EE82EFED7EC
:1012E000000000016551D8A478EF09F07AEF09F009
:1012F000C0EF09F0BC8ABC8CBC8EBB82BB84BB86B1
:10130000BB88BB8A70EF0AF0BB94BB96BB98BB9AB4
:1013100036EF0AF0BB98BB96BB94BB8A36EF0AF057
:10132000BB98BB96BB84BB9A36EF0AF0BB98BB96C2
:10133000BB84BB8A36EF0AF0BB98BB86BB94BB9AD2
:1013400036EF0AF0BB98BB86BB94BB8A36EF0AF037
:10135000BB98BB86BB84BB9A36EF0AF0BB98BB86B2
:10136000BB84BB8A36EF0AF0BB88BB96BB94BB9AA2
:1013700036EF0AF0BB88BB96BB94BB8A36EF0AF007
:1013800064C04EF04F6A516A0A0E506E52EC0BF078
:101390004F50000AD8B4CFEF09F036EF0AF04E50A4
:1013A000000AD8B484EF09F0010AD8B48AEF09F032
:1013B000030AD8B490EF09F0010AD8B496EF09F007
:1013C000070AD8B49CEF09F0010AD8B4A2EF09F0DB
:1013D000030AD8B4A8EF09F0010AD8B4AEEF09F0B7
:1013E0000F0AD8B4B4EF09F0010AD8B4BAEF09F083
:1013F00036EF0AF0BC9ABC9CBC9EBB9270EF0AF020
:10140000BC9EBC9CBC9ABB8270EF0AF0BC9EBC9C8C
:10141000BC8ABB9270EF0AF0BC9EBC9CBC8ABB82AB
:1014200070EF0AF0BC9EBC8CBC9ABB9270EF0AF0C5
:10143000BC9EBC8CBC9ABB8270EF0AF0BC9EBC8C7C
:10144000BC8ABB9270EF0AF0BC9EBC8CBC8ABB828B
:1014500070EF0AF0BC8EBC9CBC9ABB9270EF0AF095
:10146000BC8EBC9CBC9ABB8270EF0AF064C04EF08C
:101470004F6A516A0A0E506EF1EC0AF04F50000AA2
:10148000D8B445EF0AF070EF0AF04E50000AD8B415
:10149000FAEF09F0010AD8B400EF0AF0030AD8B451
:1014A00006EF0AF0010AD8B40CEF0AF0070AD8B424
:1014B00012EF0AF0010AD8B418EF0AF0030AD8B400
:1014C0001EEF0AF0010AD8B424EF0AF00F0AD8B4CC
:1014D0002AEF0AF0010AD8B430EF0AF070EF0AF0F0
:0E14E000BC86350EE82EFED70000BC9612002A
:1014F0006F0060FF4BF03901A4950001E751D8B4AB
:1015000084EF0AF086EF0AF0A2EF0AF04D6A000EAF
:101510004C6E3C0E4C24D96E010E4D20DA6EDF6A03
:101520004C4A4D2A4DBE9EEF0AF04D5009E13C0E4B
:101530004C5CD8A09EEF0AF0A0EF0AF089EF0AF009
:10154000EDEF0AF04D6A000E4C6E3C0E4C24D96E45
:10155000010E4D20DA6E4C50010FE16EE26A6F0011
:101560007FFFE7FF3C0E4C24D96E010E4D20DA6E52
:10157000DF6A4C4A4D2A4DBEC7EF0AF04D5009E1D3
:101580003C0E4C5CD8A0C7EF0AF0C9EF0AF0A5EFFB
:101590000AF03D50496E3E504A6E3D4A3E2A4ABED0
:1015A000DBEF0AF04A5009E1330E495CD8A0DBEFCB
:1015B0000AF0DDEF0AF0EDEF0AF03F50D8A4E3EFB8
:1015C0000AF0E5EF0AF0E9EF0AF0010E3F6EEAEFEC
:1015D0000AF03F6A3E6A000E3D6E60002FF1D8FFB0
:1015E00011000001616B51BEFAEF0AF0F8EF0AF04A
:1015F00000EF0BF0506C511ED8B0512A010E616FF4
:101600004FBE07EF0BF005EF0BF00DEF0BF04E6C3C
:101610004F1ED8B04F2A010E611B636B000E626F24
:1016200050505110D8B417EF0BF019EF0BF041EFF9
:101630000BF0010E606F21EF0BF0D8905036513651
:10164000602B51AE26EF0BF028EF0BF01DEF0BF0E7
:10165000D8906237633750504E5C51504F58D8A0E5
:1016600034EF0BF036EF0BF03BEF0BF050504E5ECB
:1016700051504F5A6281D89051325032602F28EF2A
:101680000BF06151D8B447EF0BF049EF0BF04DEF81
:101690000BF0626D631FD8B0632B62C04EF063C065
:1016A0004FF012000001616B4FBE5BEF0BF059EF82
:1016B0000BF061EF0BF04E6C4F1ED8B04F2A010EAD
:1016C000616F51BE68EF0BF066EF0BF06CEF0BF043
:1016D000506C511ED8B0512A50505110D8B473EFED
:1016E0000BF075EF0BF099EF0BF0010E606F7DEFD3
:1016F0000BF0D89050365136602B51AE82EF0BF084
:1017000084EF0BF079EF0BF050504E5C51504F5876
:10171000D8A08DEF0BF08FEF0BF093EF0BF0505044
:101720004E5E51504F5AD89051325032602F84EF54
:101730000BF06151D8B49FEF0BF0A1EF0BF0A5EFC8
:101740000BF04E6C4F1ED8B04F2A4EC04EF04FC01B
:101750004FF012003901A191100EE82EFED76F0054
:1017600028FF40F040500F0B416E0F0E4118D8B4C7
:10177000BCEF0BF0BEEF0BF0FAEF0BF040B8C3EF8D
:101780000BF0C5EF0BF0CDEF0BF03C0E4124D96E02
:10179000DA6A010EDA22010EDF6E40BAD2EF0BF0E8
:1017A000D4EF0BF0DCEF0BF04B0E4124D96EDA6A6C
:1017B000010EDA22010EDF6E40BCE1EF0BF0E3EF29
:1017C0000BF0EBEF0BF05A0E4124D96EDA6A010EE2
:1017D000DA22010EDF6E40BEF0EF0BF0F2EF0BF0FD
:1017E000FAEF0BF0690E4124D96EDA6A010EDA22A3
:0617F000010EDF6E110086
:1017F8006F0060FF48F03A0157AD05EF0CF007EFB6
:101808000CF03AEF0CF0579D010E0001EA6FE86BFF
:10181800010EE76F31EF0CF0090E476E1E0E466E93
:10182800E40EE82EFED7462EFCD7472EFAD700D076
:101838000001E82B140EE819D8A425EF0CF027EFC7
:101848000CF031EF0CF0010EEB6FEBC0ECF0ECC0DC
:101858003FF03FC0EDF0ACEC07F0CBAC36EF0CF04E
:1018680038EF0CF010EF0CF047EF0CF057AF3FEFEC
:101878000CF041EF0CF047EF0CF0579F010E000100
:10188800E96F010EE76F600023F1D8FF1100BC88F3
:10189800BC9ABC9CBC9EBB92BB94BB96BB98BB9AA3
:1018A800BC96BC94BC92BC900001E96BEA6BBC98F6
:1018B800350EE82EFED70000010E0001666F6000AD
:1018C8009BF1BCFF350EE82EFED700000001662B09
:1018D800070E666572EF0CF074EF0CF063EF0CF016
:1018E800050E646F010E6AEC09F04F6A050E4E6E24
:1018F8006BEC0DF0010E0001EB6FEBC03FF03FC049
:10190800ECF0ECC0EDF0EEEC05F04F6A0A0E4E6E0E
:101918006BEC0DF0050E0001646F000E6AEC09F027
:101928000001EB6BEEEC05F01200BC8ABC8CBC8E9F
:10193800BB82BB84BB86BB88BB8AE00E436E60005B
:101948000FF1BCFF350EE82EFED70000432AE60E45
:101958004364B1EF0CF0B3EF0CF0A3EF0CF000010F
:10196800EDB102D0BB9201D0BB820001ECB102D034
:10197800BC9E01D0BC8E3FB002D0BC9C01D0BC8CB8
:101988000001EBB102D0BC9A01D0BC8A350EE82E1A
:10199800FED700006F0030FF42F04280428242844E
:1019A80060000BF1BCFF1200BC9ABC9CBC9EBB92B1
:1019B800BB94BB96BB98BB9A436A60000FF1BCFF0F
:1019C800350EE82EFED70000432A060E4364EFEFDB
:1019D8000CF0F1EF0CF0E1EF0CF00001EDB102D0EA
:1019E800BB9201D0BB820001ECB102D0BC9E01D0F9
:1019F800BC8E3FB002D0BC9C01D0BC8C0001EBB1C6
:101A080002D0BC9A01D0BC8A350EE82EFED7000061
:101A18006F0030FF42F042804282428460000BF146
:101A2800BCFF1200200EF66E1B0EF76E000EF86E4D
:101A380000EE78F110EE3CF009006F00D7FFEEFFE2
:101A4800E550E150F9E100EE00F1780EEE6AE806A3
:101A5800FDE100EEE7F0080EEE6AE806FDE100EEB3
:101A680001F03F0EEE6AE806FDE1080ED56E000EA5
:101A7800D66E000ED76E000EF86E000101EF04F06E
:101A88006F0060FF44F03901A39F0001ED51D8B405
:101A980050EF0DF052EF0DF063EF0DF0ED6BEE51DE
:101AA800D8A459EF0DF05BEF0DF05FEF0DF099EC56
:101AB8000CF067EF0DF0ACEC07F067EF0DF0010EDE
:101AC800ED6FD8EC0CF0600013F1D8FF11000001A5
:101AD800616B000E606F80EF0DF0090E516E1E0EE7
:101AE800506EE40EE82EFED7502EFCD7512EFAD7B2
:101AF80000D00001604B612B60514E5C4F50800A52
:101B0800506E6151800A5058D8B08DEF0DF08FEFAC
:101B18000DF071EF0DF0120008090A070D0E0B0306
:101B28000405060102001B0C181C1D251A141917A0
:101B3800161510110F2B2C242A13121E231F2928C7
:101B480027263A203B363922212E2F373830313597
:061B58002D3433321100B0
:020000040020DA
:10000000FF0FFF0FFF0FFF0FFF0FFF0FFF0FFF0F80
:020000040030CA
:0A0000008CFFFFFF9FFFFFFFFFFFD3
:00000001FF
